:020000000C28CA
:10000800FF000308F7000408F8000A08F90062284E
:100018006120E7006020E6005F20E5005E20E40044
:100028005D20E3005C20E2005B20E1005A20E00054
:100038005920DF005820DE00E801E901EA01EB0160
:10004800EC01ED01EE01282883168101C0308312EE
:100058008B00033083168C00F03083129000EC0183
:100068005E08F3005E08EF005E08A0005E08F0007E
:100078000830920007309F008316920101308312E6
:100088009100F201F20A8316850186018312850028
:100098008601EB01F101F10AEC016810E810EA01B0
:1000A800C421121510145728C034F934A434B034BC
:1000B800993492348234F83480349034831603139C
:1000C8008C1CA22883128C1CA2288C109228023027
:1000D800F2006A0885006F0886006A08023E9028C8
:1000E8000430F2006A088500200886006A08043E89
:1000F80090280830F2008A28F201F20A6A0885007E
:10010800730886006A0A9028F201F20A6A088500D4
:10011800700886006A08083E8500A2287208003A1E
:1001280003198828013A03196B28033A031974281C
:10013800063A03197D280C3A0319802883160C1CEB
:10014800502983120C1C50290C10DC308E000B3007
:100158008F00681CD128EC03EB08031DBD28F108AB
:10016800031DBD28EC08031DBD286810EA012F22D5
:10017800492978306C02031CD1287730EC00F10350
:100188003C307102031CD1283B30F100EB030C30EA
:100198006B02031CD1280B30EB00E81CD528E810B3
:1001A800D628E8148316FF308500860083120618C7
:1001B800F028681CE2286810EA01E5286814103065
:1001C800EA00F930F6006400F60BE728EB28640033
:1001D80083120313061CEC2868184C2983168C100C
:1001E8008312061A0B2906190029EB0A0C306B0238
:1001F800031C4929EB014929F10A3C307102031C0F
:100208000B29F101EB0A0C306B020318EB0186197C
:100218001D29861C4229F1033C307102031C1D294B
:100228003B30F100EB030C306B02031C1D290B3033
:10023800EB0006193129EC0AEC0A78306C02031C31
:100248003129EC01F10A3C307102031C3129F1011A
:10025800EB0A0C306B020318EB0186184929EC03F2
:10026800EC0378306C02031C49297730EC00F10369
:100278003C307102031C49293B30F100EB030C3080
:100288006B02031C49290B30EB00362283168C14B1
:10029800831685018601592179088A007808840027
:1002A80077088300FF0E7F0E09008312F001A0017A
:1002B800EF01F301FB01FA01EB08031D9429710812
:1002C800FA000A307A02031C6D290A30FA02F00A91
:1002D800652970085E3E831384000008F0007A08E0
:1002E8005E3E84000008A0006818E81C7D29803064
:1002F800A00203106C0CFB000A307B02031C882947
:100308000A30FB02EF0A80296F085E3E83138400DF
:100318000008EF007B085E3E84000008F300080038
:100328007108FA000A307A02031C9E290A30FA0280
:10033800EF0A96296F085E3E831384000008EF00D9
:100348007A085E3E84000008F3006B08FB000A3060
:100358007B02031CB3290A30FB02F00AAB297008A0
:100368005E3E831384000008F0007B085E3E840034
:100378000008A0006818E81C08008030A0020800E7
:100388008312F001A001EF01F301F401F501EB087C
:10039800031DFF297108F5000A307502031CD829CE
:1003A8000A30F502F00AD02970085E3E83138400F3
:1003B8000008F00075085E3E84000008A000681878
:1003C800E81CE8298030A00203106C0CF4000A3005
:1003D8007402031CF3290A30F402EF0AEB296F08B0
:1003E8005E3E831384000008EF0074085E3E8400BC
:1003F8000008F30008007108F5000A307502031CB4
:10040800092A0A30F502EF0A012A6F085E3E8313B3
:1004180084000008EF0075085E3E84000008F300C1
:100428006B08F4000A307402031C1E2A0A30F40216
:10043800F00A162A70085E3E831384000008F00054
:1004480074085E3E84000008A0006818E81C0800D4
:100458008030A00208006908EB006E08F1006D0802
:10046800EC0008006B08E9007108EE006C08ED006C
:0204780008007A
:02400E00783FF9
:00000001FF
